:0200000480007A
:100000006F008004732F2034930F80006308FF0378
:10001000930F90006304FF03930FB0006300FF038E
:10002000130F000063040F0067000F00732F2034CC
:1000300063540F006F00400093E19153171F0000BD
:1000400023223FFC6FF09FFF93000000130100008C
:10005000930100001302000093020000130300004C
:100060009303000013040000930400001305000034
:10007000930500001306000093060000130700001C
:100080009307000013080000930800001309000004
:1000900093090000130A0000930A0000130B0000EC
:1000A000930B0000130C0000930C0000130D0000D4
:1000B000930D0000130E0000930E0000130F0000BC
:1000C000930F0000732540F16310050097020000B4
:1000D000938202017390523073500018970200000F
:1000E0009382020273905230B70200809382F2FF33
:1000F0007390023B9302F0017390023A73504030C8
:100100009702000093824201739052307350203066
:100110007350303093010000970200009382C2EECA
:1001200073905230130510001315F501634C050050
:100130000F00F00F930110009308D0051305000085
:100140007300000093020000638A02007390521053
:10015000B7B2000093829210739022307350003037
:10016000970200009382420173901234732540F18C
:100170007300203093012000930000001301100051
:1001800063E620006312302E63163000E3EE20FE9B
:10019000631C302C930130009300E0FF1301F0FF4B
:1001A00063E620006312302C63163000E3EE20FE7D
:1001B000631C302A93014000930000001301F0FFFC
:1001C00063E620006312302A63163000E3EE20FE5F
:1001D000631C3028930150009300100013010000AD
:1001E00063E420006314300063103028E3EE20FE47
:1001F000930160009300F0FF1301E0FF63E420002F
:100200006314300063123026E3EE20FE9301700089
:100210009300F0FF1301000063E42000631430003A
:1002200063143024E3EE20FE93018000B7000080C9
:10023000370100801301F1FF63E4200063143000F4
:1002400063143022E3EE20FE9301900013020000BD
:10025000B70000F0370100F01301F1FF63E6202042
:100260001302120093022000E31452FE9301A00037
:1002700013020000B70000F0370100F01301F1FF96
:100280001300000063E2201E1302120093022000FC
:10029000E31252FE9301B00013020000B70000F019
:1002A000370100F01301F1FF1300000013000000FC
:1002B00063EC201A1302120093022000E31052FE96
:1002C0009301C00013020000B70000F0130000000B
:1002D000370100F01301F1FF63E820181302120048
:1002E00093022000E31252FE9301D000130200009B
:1002F000B70000F013000000370100F01301F1FF18
:100300001300000063E22016130212009302200083
:10031000E31052FE9301E00013020000B70000F06A
:100320001300000013000000370100F01301F1FF7B
:1003300063EC20121302120093022000E31052FE1D
:100340009301F00013020000B70000F0370100F045
:100350001301F1FF63EA2010130212009302200040
:10036000E31452FE9301000113020000B70000F0F5
:10037000370100F01301F1FF1300000063E6200EC7
:100380001302120093022000E31252FE93011001A7
:1003900013020000B70000F0370100F01301F1FF75
:1003A000130000001300000063E0200C1302120091
:1003B00093022000E31052FE93012001130200007B
:1003C000B70000F013000000370100F01301F1FF47
:1003D00063EC20081302120093022000E31252FE85
:1003E0009301300113020000B70000F01300000079
:1003F000370100F01301F1FF1300000063E620064F
:100400001302120093022000E31052FE93014001F8
:1004100013020000B70000F01300000013000000FA
:10042000370100F01301F1FF63E020041302120012
:1004300093022000E31052FE93001000636A100044
:100440009380100093801000938010009380100020
:1004500093801000938010009303300093015001AB
:1004600063947000631030020F00F00F638001008E
:100470009391110093E111009308D00513850100B9
:10048000730000000F00F00F930110009308D005D7
:100490001305000073000000731000C0000000008E
:1004A000000000000000000000000000000000004C
:0C04B00000000000000000000000000040
:1010000000000000000000000000000000000000E0
:1010100000000000000000000000000000000000D0
:1010200000000000000000000000000000000000C0
:1010300000000000000000000000000000000000B0
:081040000000000000000000A8
:040000058000000077
:00000001FF
